 gpiosdk

 Timestamp is 4da293d0 (Mon Apr 11 17:38:24 2011)

 Preferred load address is 10000000

 Start         Length     Name                   Class
 0001:00000000 00000004H .CRT$XCA                CODE
 0001:00000004 00000004H .CRT$XCZ                CODE
 0001:00000008 00000004H .CRT$XIA                CODE
 0001:0000000c 00000004H .CRT$XIZ                CODE
 0001:00000010 00000004H .CRT$XPA                CODE
 0001:00000014 00000004H .CRT$XPZ                CODE
 0001:00000018 00000004H .CRT$XTA                CODE
 0001:0000001c 00000004H .CRT$XTZ                CODE
 0001:00000020 00000028H .rdata                  CODE
 0001:00000048 00000024H .rdata$debug            CODE
 0001:0000006c 00000674H .text                   CODE
 0001:000006e0 00000014H .xdata                  CODE
 0001:000006f4 00000014H .idata$2                CODE
 0001:00000708 00000014H .idata$3                CODE
 0001:0000071c 0000002cH .idata$4                CODE
 0001:00000748 0000000cH .idata$6                CODE
 0001:00000760 000001a5H .edata                  CODE
 0002:00000000 0000002cH .idata$5                DATA
 0002:00000030 00000450H .data                   DATA
 0002:00000480 00000010H .bss                    DATA
 0003:00000000 000000e0H .pdata                  DATA

  Address         Publics by Value              Rva+Base       Lib:Object

 0000:00000000       ___safe_se_handler_count   00000000     <absolute>
 0000:00000000       ___safe_se_handler_table   00000000     <absolute>
 0001:00000000       __xc_a                     10001000     corelib0:crt0init.obj
 0001:00000004       __xc_z                     10001004     corelib0:crt0init.obj
 0001:00000008       __xi_a                     10001008     corelib0:crt0init.obj
 0001:0000000c       __xi_z                     1000100c     corelib0:crt0init.obj
 0001:00000010       __xp_a                     10001010     corelib0:crt0init.obj
 0001:00000014       __xp_z                     10001014     corelib0:crt0init.obj
 0001:00000018       __xt_a                     10001018     corelib0:crt0init.obj
 0001:0000001c       __xt_z                     1000101c     corelib0:crt0init.obj
 0001:0000003c       ??_C@_1M@BPKHPEKM@?$AAG?$AAP?$AAI?$AA1?$AA?3?$AA?$AA@ 1000103c     gpiosdk.obj
 0001:0000006c       DllMain                    1000106c f   gpiosdk.obj
 0001:00000080       GpioInit                   10001080 f   gpiosdk.obj
 0001:000000e8       GpioDeinit                 100010e8 f   gpiosdk.obj
 0001:00000298       GpioGetConfig              10001298 f   gpiosdk.obj
 0001:000002a8       GpioSetConfig              100012a8 f   gpiosdk.obj
 0001:000002b8       GpioReadPin                100012b8 f   gpiosdk.obj
 0001:000002c8       GpioWritePin               100012c8 f   gpiosdk.obj
 0001:000002d8       GpioReadPort               100012d8 f   gpiosdk.obj
 0001:000002e8       GpioWritePort              100012e8 f   gpiosdk.obj
 0001:000002f8       GpioReadIntrPin            100012f8 f   gpiosdk.obj
 0001:00000308       GpioReadIntrPort           10001308 f   gpiosdk.obj
 0001:00000318       GpioClearIntrPin           10001318 f   gpiosdk.obj
 0001:00000328       GpioClearIntrPort          10001328 f   gpiosdk.obj
 0001:00000338       GpioRegisterEvent          10001338 f   gpiosdk.obj
 0001:00000348       GpioDeregisterEvent        10001348 f   gpiosdk.obj
 0001:00000358       GpioGetEvent               10001358 f   gpiosdk.obj
 0001:00000368       DisableThreadLibraryCalls  10001368 f   coredll:COREDLL.dll
 0001:00000378       CreateFileW                10001378 f   coredll:COREDLL.dll
 0001:00000388       CloseHandle                10001388 f   coredll:COREDLL.dll
 0001:00000398       SetLastError               10001398 f   coredll:COREDLL.dll
 0001:000003a8       DeviceIoControl            100013a8 f   coredll:COREDLL.dll
 0001:000004b0       _DllMainCRTStartup         100014b0 f   corelib0:pegdmain.obj
 0001:0000059c       _cexit                     1000159c f   corelib0:cexit.obj
 0001:000005ac       _initterm                  100015ac f   corelib0:crt0dat.obj
 0001:000005d8       _cinit                     100015d8 f   corelib0:crt0dat.obj
 0001:00000638       __security_init_cookie     10001638 f   corelib0:seccinit.obj
 0001:00000684       __crt_ExitProcess          10001684 f   corelib0:exitproc_proxy.obj
 0001:00000690       _XcptFilter                10001690 f   corelib1:COREDLL.dll
 0001:000006a0       __C_specific_handler       100016a0 f   corelib1:COREDLL.dll
 0001:000006b0       free                       100016b0 f   corelib1:COREDLL.dll
 0001:000006c0       __security_gen_cookie2     100016c0 f   corelib1:COREDLL.dll
 0001:000006d0       TerminateProcess           100016d0 f   coredll:COREDLL.dll
 0001:000006f4       __IMPORT_DESCRIPTOR_COREDLL 100016f4     coredll:COREDLL.dll
 0001:00000708       __NULL_IMPORT_DESCRIPTOR   10001708     coredll:COREDLL.dll
 0002:00000000       __imp_DisableThreadLibraryCalls 10002000     coredll:COREDLL.dll
 0002:00000004       __imp_CreateFileW          10002004     coredll:COREDLL.dll
 0002:00000008       __imp_CloseHandle          10002008     coredll:COREDLL.dll
 0002:0000000c       __imp_SetLastError         1000200c     coredll:COREDLL.dll
 0002:00000010       __imp_DeviceIoControl      10002010     coredll:COREDLL.dll
 0002:00000014       __imp__XcptFilter          10002014     corelib1:COREDLL.dll
 0002:00000018       __imp___C_specific_handler 10002018     corelib1:COREDLL.dll
 0002:0000001c       __imp_free                 1000201c     corelib1:COREDLL.dll
 0002:00000020       __imp___security_gen_cookie2 10002020     corelib1:COREDLL.dll
 0002:00000024       __imp_TerminateProcess     10002024     coredll:COREDLL.dll
 0002:00000028       \177COREDLL_NULL_THUNK_DATA 10002028     coredll:COREDLL.dll
 0002:00000030       ?dpCurSettings@@3U_DBGPARAM@@A 10002030     DebugZones.obj
 0002:00000478       __security_cookie          10002478     corelib0:seccinit.obj
 0002:0000047c       __security_cookie_complement 1000247c     corelib0:seccinit.obj
 0002:00000480       _exitflag                  10002480     corelib0:cexit.obj
 0002:00000484       __onexitend                10002484     <common>
 0002:00000488       __onexitbegin              10002488     <common>
 0002:0000048c       _pRawDllMain               1000248c     <common>

 entry point at        0001:000004b0

 Static symbols

 0001:00000124       ?CallDriver@@YAHHPAUGPIO_CONFIG@@@Z 10001124 f   gpiosdk.obj
 0001:000001b8       ?CallDriver@@YAHHPAUGPIO@@@Z 100011b8 f   gpiosdk.obj
 0001:00000228       ?CallDriver@@YAHHPAUGPIO_EVENT@@@Z 10001228 f   gpiosdk.obj
 0001:000003c0       _DllMainCRTStartupHelper   100013c0 f   corelib0:pegdmain.obj
 0001:000004dc       doexit                     100014dc f   corelib0:cexit.obj
